:10000000A5C21895189518951895189518951895CE
:100010005FC4BCC318951895189518951895189530
:1000200018951895189500000203030102000103BA
:1000300002000101010003030002030103000303A6
:100040000202010103000103020001030300030196
:10005000020201030300030102020303030003037E
:100060000200010101000303020203030300030372
:10007000020201030300000101000301010000006E
:100080000000020303010200020202020002030058
:10009000020202020202030002020200000001004A
:1000A0000200020202020300020002020002030038
:1000B000000202000002030002020202000003002C
:1000C0000202000202000300000202000000010020
:1000D0000202020202020000000202000000000010
:1000E00002020002020002000202020200000200FC
:1000F00000020200000202000200020200020200EE
:1001000002000202020202000202020000000000DD
:1001100002020202020202000202020200020200C5
:1001200002030302020200000003030000000000BB
:1001300002030102020002000203030200000200A7
:100140000003030000020200020103020002020099
:100150000201030202020200020303000000000089
:100160000203030202020200020303020002020071
:100170000303020303020100010302010100010065
:100180000303000303000300030302030100030051
:100190000103020101020300030102030102030043
:1001A0000301020303020300030302010100010033
:1001B000030302030302030003030203010203001B
:1001C0000303030302020100010303010000010015
:1001D0000303010302000300030303030000030001
:1001E00001030301000203000301030300020300F3
:1001F00003010303020203000303030100000100E3
:1002000003030303020203000303030300020300CA
:1002100002030302020301000003030000010100C6
:1002200002030102020103000203030200010300B2
:1002300000030300000303000201030200030300A4
:100240000201030202030300020303000001010094
:10025000020303020203030002030302000303007C
:100260000302030302030100010203010001010074
:100270000302010302010300030203030001030060
:100280000102030100030300030003030003030052
:100290000300030302030300030203010001010042
:1002A000030203030203030003020303000303002A
:1002B00000010100030101000000AF92BF92A09075
:1002C000700008E0B02EA69410F4ADD001C0A7D005
:1002D000BA94C9F7BF90AF900895AF92BF9281D002
:1002E00000E0109171000117E8F10CEC0093700030
:1002F000E4DF0EEB00937000E0DF00E0009372009B
:100300000093730008E0B02E0091720006950093F0
:100310007200B89A91D0B8988FD08ED08DD08CD0F2
:10032000B09B05C00091720000680093720021D05C
:10033000BA9451F708E0B02E00917300069500932F
:100340007300B89A79D0B89877D076D075D074D039
:10035000B09B05C00091730000680093730009D042
:10036000BA9451F7BF90AF90089562D061D060D039
:1003700008955ED05DD00895F8DFF7DFF6DFF5DF92
:10038000F4DFF3DFF2DFF1DFF0DFEFDF08952F932B
:1003900028D000E0109171000117B0F00CEC009330
:1003A00070008BDF04E40093700087DF20E010E032
:1003B000B89A42D0B89840D03FD03ED02A9511F498
:1003C0001A9521F0B09BF4CF2F91089504E000938B
:1003D00071002F9108952CD02BD005E20A95F1F7EA
:1003E000089500E000937100B09904C001E000930B
:1003F0007100089500E000937100C098B89ABCDFC6
:10040000B898B7DFB09B04C002E000937100089574
:10041000ACDFB09903C003E0009371000895B89A6F
:10042000DADFB8980895B89A07D0B898D4DF08955D
:100430000AEA0A95F1F708950FE00A95F1F7089591
:1004400000917100003009F480C00091710001300A
:10045000A1F401E00093600002E0009361000093CA
:10046000620001E000936300009364000093650064
:10047000009366000093670068C00091710002302D
:10048000C1F403E00093600002E00093610000E02B
:100490000093620003E0009363000093640001E0B6
:1004A0000093650003E00093660001E0009367009D
:1004B0004CC0009171000330B9F403E00093600078
:1004C00002E0009361000093620003E00093630088
:1004D00001E0009364000093650003E00093660070
:1004E00001E00093670031C0009171000430B1F465
:1004F00001E00093600002E000936100009362005D
:1005000001E0009363000093640003E00093650042
:100510000093660001E00093670017C001E00093BC
:10052000600000E0009361000093620001E000932E
:10053000630003E00093640001E00093650003E0C2
:100540000093660001E00093670008950FE50DBF7A
:1005500004E00EBF03E003BF00E00FBD03E00EBDEB
:1005600005E009BFA09AA19AA89AA99A0FEF01BB2A
:1005700000E002BBAB9AA39A00916B000860009365
:100580006B00C19AB99800E00093690000916B007C
:10059000016000936B0040E003E000936000009373
:1005A0006100009362000093630000936400009375
:1005B000650002E00093660001E00093670039D116
:1005C0000091740000936C0066D28DD201E000931C
:1005D00068007894009168000030E1F7F894A89AD8
:1005E000A99A00916B000D7F00936B00D0DE009103
:1005F0007100003011F024DF09C06FDE009171003E
:10060000003011F01DDF02C0C5D11CD1789407E085
:100610000093680000916A00023009F466C00091FE
:1006200068000030B9F7DACF80916D008B3008F0A8
:100630008AE0E6E2F0E0FEC100916D0003950093D0
:100640006D0000916D00013020F401E000936D0019
:1006500008C009E010916D00011718F401E0009343
:100660006D00089500916F00003081F000E000936C
:100670006F00089500916B00077F00936B00089551
:1006800000916B00086000936B00089501E00093F7
:100690006F00089502E0009360000093610000E0A5
:1006A000009362000093630002E0009364000093F3
:1006B00065000093660001E000936700089502E082
:1006C0000093600000E0009361000093620002E08C
:1006D00000936300009364000093650000E00093C2
:1006E000660001E000936700089500E000936A004F
:1006F00000916B00026000936B009BD0009174002E
:1007000000936C00C8D186D100917400043009F4C4
:10071000C1DF00917400033009F4D1DF00E10093E0
:10072000680000916A00023071F0009168000030AA
:10073000C1F779CF03E210917400011718F403E0B8
:1007400000937400089500E000936A0004E10093B0
:10075000680000916A000130A1F00091680000304B
:10076000C1F700917400043009F4FCC000917400DA
:10077000033009F4C1C1CED00091740000936C0025
:1007800052CF00E000936A0091D0BDCF0F930FB716
:100790000F931F93E8ECF8E0E40F10E0F11F0491D1
:1007A00002BBC0E6D0E0C40F10E0D11F1881109545
:1007B00010FB05B300F905BB11FB05B301F905BB3F
:1007C00000916B0001FF04C0473011F4A89AA9986A
:1007D0004395483008F0442700916900003031F01B
:1007E000009169000A95009369001EC0B19B0DC07D
:1007F00000916B0000FD18C000916B000160009338
:100800006B0001E000936A000CC000916B0000FFD8
:100810000BC000916B000E7F00936B0002E0009311
:100820006A0008E2009369001F910F910FBF0F91BA
:10083000189510E01EBB10E01FBBE09A0DB30093AB
:100840007400089500916F000030E9F00091740089
:1008500007FD13C000916C0010917400011738F06F
:1008600010916C0000917400011738F00895009108
:100870006B00086000936B00089500916B00077F88
:1008800000936B0008950091740007FDF9CE00916C
:100890006C0010917400011708F4ECCE10916C00FC
:1008A00000917400011708F4EBCE089500917400D4
:1008B00003950093740000917400033008F03ACF60
:1008C00003E0009374003ECF010204081020408032
:1008D0000F930FB70F9300916800003029F000913B
:1008E00068000A950093680000916B0003FF02C046
:1008F000AB9A08C000916E000A9500936E0009F053
:1009000047C0AB9800916D0000936E000F910FBF30
:100910000F91189510E01EBB10E01FBBE09A5DB36D
:1009200010917400511759F00091740010E01EBB33
:1009300010E01FBB0DBBE29AE19AE199FECF08954A
:1009400000E000936A0004E10093680000916A00EF
:10095000013009F4ADC0009168000030B9F7ADD0A6
:100960009AD061CE00E000936A0000916B000860AD
:1009700000936B0090D058DE00E100936800009176
:100980006A000230E9F2009168000030C1F7E8CF58
:10099000AB9ABCCF0091720004FB0091740000F987
:1009A000009374000091720005FB0091740001F93E
:1009B000009374000091720006FB0091740002F92C
:1009C000009374000091720007FB0091740003F91A
:1009D000009374000091730000FB0091740004F90F
:1009E000009374000091730001FB0091740005F9FD
:1009F000009374000091730002FB0091740006F9EB
:100A0000009374000091730003FB0091740007F9D8
:100A100000937400809174000AE0800F00917400CC
:100A200007FF03C087FF01C080E0873408F086E439
:100A3000E0E8F0E0E80F10E0F11FE80F10E0F11F30
:100A4000E80F10E0F11FE80F10E0F11FE80F10E0D1
:100A5000F11FE80F10E0F11FE80F10E0F11FE80FA1
:100A600010E0F11F05910093600005910093610073
:100A70000591009362000591009363000591009336
:100A80006400059100936500059100936600049150
:100A900000936700089511E01EBB10E01FBBE09AB1
:100AA0000DB300936D0000916D0000936E000895EA
:100AB00000E000936A00C0DD5ECF11E01EBB10E0D5
:100AC0001FBBE09A5DB310916D00511759F0009172
:100AD0006D0011E01EBB10E01FBB0DBBE29AE19A56
:100AE000E199FECF089512E01EBB10E01FBBE09A13
:100AF0000DB300936F00089500E000936A00009129
:100B00006B00086000936B00EEDF2AD000E10093D9
:100B1000680000916A00023029F0009168000030FE
:100B2000C1F710C000E000936A0004E10093680080
:100B300000916A00013009F444C00091680000305F
:100B4000B9F702D0D0DF6FCD00916F0012E01EBB6D
:100B500010E01FBB0DBBE29AE19AE199FECF089528
:100B600000916F000030B9F001E00093600002E0F6
:100B7000009361000093620001E00093630003E0D2
:100B8000009364000093650002E00093660001E0BA
:100B900000936700089503E00093600000E0009375
:100BA00061000093620003E000936300009364001F
:100BB0000093650000E00093660001E00093670089
:0C0BC000089500E000936A004DDD9FCF17
:00000001FF
